:10000000C00C0020C5000000C1000000C1000000BD
:1000100000000000000000000000000000000000E0
:10002000000000000000000000000000C10000000F
:100030000000000000000000C1000000C10000003E
:10004000C1000000C1000000C1000000C1000000AC
:10005000C1000000C1000000C1000000C10000009C
:10006000C1000000C1000000C1000000C10000008C
:10007000C1460000C9450000C1000000C1000000E9
:10008000C1000000C1000000C1000000C10000006C
:10009000C1000000C1000000C1000000C10000005C
:1000A000C1000000C1000000C1000000C10000004C
:1000B000C1000000C1000000C1000000C10000003C
:1000C000FEE7C04610B5154B154A9A420ED2154BA5
:1000D000124A0332D21A92080132920000231048C9
:1000E0001149CC58C45004339342FAD10F4B104AF3
:1000F0009A420ED20F4B0D490331C91A89080131BA
:1001000089000023140000201A19106004338B4268
:10011000FAD104F00DFC02F0EDFD10BD0C00002042
:100120000000002004000020DC4D0000C00800207A
:100130000C0000201000002070B584B004006A4656
:100140000E4B694661CB61C11B680B600C4B1B6891
:1001500001930C494B699B019B0F9B00985889693F
:100160000905090F013104F02FFC4000210004F0C3
:100170002BFC01304008023804B070BD004D000077
:10018000000000200002005001220A4B1A700022D9
:100190000949180053009B189B00CB189B7ADB077A
:1001A00003D503780133DBB203700132202AF1D189
:1001B0007047C046A4040020A80400200F23034079
:1001C00018003730092B01D8303318007047C0466B
:1001D0000022C30700D55E32830701D5BC235A40F5
:1001E000430701D561235A40030701D5C2235A4072
:1001F000C30601D59D235A40830601D523235A40C7
:10020000430601D546235A4043B2002B01DA8C2322
:100210005A4010007047C04630B5154B1B78002B74
:1002200005D0144B1B780020002B09D119E0124B8C
:100230001B78692B1BD0104B1B78492BF1D116E092
:100240000E4A802109040C4D0A4C93690B42FCD1E3
:100250002B5CDBB213600130C0B22378DBB2834287
:10026000F3D80022034B1A700132054B1A6030BDDF
:1002700076060020B1010020BC01002000000540EE
:100280009442005070B5114B1B78002B1DD1104BC0
:100290001B78002B13D000200E4A802109040E4C3D
:1002A00000260B4D93690B42FCD1235CDBB213603B
:1002B00026540130C0B22B78DBB28342F2D8002240
:1002C000034B1A700132054B1A6070BDF802002012
:1002D000B1010020000005408C0000209442005035
:1002E000184B1B78002B2CD1420883085340434005
:1002F000C208534002095340420953408209534007
:10030000C209534001221340DB011818C0B20E4944
:10031000802212048B691342FCD10B4BDA68102146
:100320008A43DA60D96820220A43DA60D968082251
:100330000A43DA6018601900802252058B69134263
:10034000FCD070479801002000001540F0B55F46D2
:1003500056464D464446F0B491B0444B5D78EDB2FC
:10036000EB1E0020392B79D82C1D002200233F489A
:10037000815C6E46B1540133DBB21A1EA242F7DB38
:10038000AF1C01240020394E335D5840C0B2FFF746
:100390001FFF0134A742F7D12B006B44987003353F
:1003A000012D43DD012300210122314883463148DC
:1003B0008246D946D0465F46D4466846C05CFE2891
:1003C0000FD148460078C0184018FD2446463454E2
:1003D0000131C9B248460078C01840181F3C345457
:1003E00017E0FD280FD122480078C0184018FD24DE
:1003F000204E34540131C9B21D480078C01840184D
:10040000203C345405E05C462478E41864185646D1
:1004100030553878C3185B18053300206446E05423
:100420000132D2B2131EAB42C7DB02E0012300212E
:1004300001220F480478E4B20E4DFE262E550478B2
:10044000E3185B18EE5403780133D2188918C9B247
:1004500001700122084B1A600078C0B211B03CBC98
:1004600090469946A246AB46F0BDC046BC0100206E
:10047000B10100208C00002094420050F0B55F468E
:1004800056464D464446F0B485B0E14B1B78002BF0
:1004900007D0E04B1B78002B03D0FFF7F3FE00F0F2
:1004A000C0FCDD4B1B78002B00D117E2DB4B1B7827
:1004B000002B00D192E001270024002500230193A6
:1004C000D74B9846D74B9946220000E00F007C1E80
:1004D000E4B26300D449595A4046185A4140404654
:1004E00019521B5A9BB2002B03D1D04B1B78002B07
:1004F0006AD0019B0133DBB20193CD4B1B78002BFB
:1005000048D06E0076197600F31C9A46601C0011E4
:10051000C0B2FFF753FE4B4652469854331D9A46DD
:100520003800FFF74BFE4B46524698546400BE4BD2
:10053000E35A1B0A9A46731D9B4653461809FFF758
:100540003DFE4B465A469854B31D9B465046FFF716
:1005500035FE4B465A469854B34BE45AE4B2F31D69
:100560009A462009FFF72AFE4B4652469854082324
:100570009A46B2442000FFF721FE4B46524698545B
:1005800009360D234A4693556A1C5300D21852006F
:10059000D2B217E06B005B199A1CA2498F54D91C88
:1005A0006400A14AA25A120A9E484254191D9E4A4A
:1005B000A25AD2B2425405330D22C2546A1C5300CF
:1005C000D218D2B20135EDB2944B1B78DBB2791C54
:1005D000C9B2BB4200D979E7140002E0002400232D
:1005E00001938E4B5B78002B00D1A0E0002000230C
:1005F000994600258F4B9A46A0462C006B008E4AE8
:100600009A5A5146595A4A4051465A525B5A9BB2DD
:10061000002B03D1854B1B78002B6DD0019B013340
:10062000DBB201937D4B1E780136AE19F6B2804BDA
:100630001B78002B42D04B465F004F447F00FB1CD1
:1006400043449B463009FFF7B9FD764B5A46985410
:100650003B1D43449B463000FFF7B0FD714B5A46AB
:10066000985463009B46744B5A46D65A360A7C1DF2
:1006700044443009FFF7A2FD6A4B1855BC1D4444A1
:100680003000FFF79BFD674B18556B4B5A46D45A09
:10069000E4B2FE1D46442009FFF790FD614B9855DA
:1006A0003E00083646442000FFF788FD5D4B985514
:1006B000093747440D235B4AD35518E04B465B008E
:1006C0004B449A1C424457498E54DA1C42446400FD
:1006D0005949615A090A534881541A1D42445649DE
:1006E000615AC9B28154053343440D22C2544B466A
:1006F0000133DBB2994601200135EDB2474B5B78FF
:10070000DBB2AB4200D978E7444600280FD0484B13
:100710001B78002B06D04B465B004B445B00E41873
:10072000E4B204E04B465B004B44E418E4B23B4BBC
:100730009B78002B00D1AAE00023994600263F4B6E
:100740009A46A046340073003D4A9A5A5146595A77
:100750004A4051465A525B5A9BB2002B04D1334B4C
:100760001B78002B00D18AE0019B0133DBB201939F
:100770002A4B1B78294A5578ED1801357519EDB2C9
:100780002B4B1B78002B5DD04B465F004F447F0006
:10079000FB1C43449B462809FFF710FD214B5A469A
:1007A00098543B1D43449B462800FFF707FD1D4B13
:1007B0005A46985463009B46214B5A46D55A2D0AF7
:1007C0007C1D44442809FFF7F9FC164B1855BC1D45
:1007D00044442800FFF7F2FC124B1855184B5A46B8
:1007E000D45AE4B2FD1D45442009FFF7E7FC0D4B48
:1007F00058553D00083545442000FFF7DFFC094B04
:100800005855093747440D23064AD35533E0C046AF
:10081000B1010020A5040020F8020020B80100204A
:100820007C060020BC010020540100203E03002073
:10083000CD000020D000002064030020080200202A
:10084000340600204B465B004B449A1C4244D4497A
:100850008D54DA1C42446400D249615A090AD048D6
:1008600081541A1D4244CF49615AC9B2815405339B
:1008700043440D22C2544B460133DBB29946013644
:10088000F6B2C94B9B78DBB2B34200D95AE7C74BEB
:100890001B78002B12D0019D2809FFF78FFCC04C5C
:1008A00060702800FFF78AFCA0706B00AC466344C0
:1008B0005B000433DBB2BE4A137009E0B84B019908
:1008C00059700B0001335A009B18DBB2B84A137001
:1008D000FFF7A2FC0022B74B1A70A2E2B64B1B78BE
:1008E000002B00D19DE2B54B1B78002B00D198E284
:1008F000B34B1B78002B00D193E2B24B1B78002B3B
:1009000000D18BE22027402660250024A64B984684
:10091000AC4B9B4643461B785A461278DBB2934257
:1009200000D9B8E0A1466200A74BD35AA749525A52
:100930005A40102300210120104201D00131C9B2D8
:100940005208013BDBB2002BF6D1A14B1B78002BE8
:1009500006D0A04B1A680123484683401A4201D1B1
:10096000012938D98E4BFE221A70F63A5A709F70C0
:100970000022DA70984A94464946525CD2B29246B6
:10098000511CC9B260464A46815452461A71A2228D
:100990005A7100229A711022DA718C494A4650002D
:1009A000425AD2B21A72425A120A5A72FFF7CEFC57
:1009B0007F4B1870894B1B78002B09D085490A683A
:1009C00001234846834013430B600022844B1A8066
:1009D000FFF758FC5FE04B465B007B4A9A5A7B4925
:1009E000585A504057D08446C30712D401220123DD
:1009F0009A460194010008001041544604420BD16C
:100A00000133DBB20132102BF5D103936046019C18
:100A100005E00023039302E003936046019CFE215E
:100A20005F4B1970F93959709F700021D9706A496C
:100A30008A464B46C95CCBB2019301336A46D372F6
:100A4000D37A9C465346494662465A54544A6B46AA
:100A50001B7913714A005D49525A1040421E904161
:100A6000A122101A4E4A50716B461B7B9371FFF7FF
:100A70006DFC4F4B1870594B1B78002B09D0554912
:100A80000A6801234846834013430B600022544BFD
:100A90001A80FFF7F7FB444B5B784A4A1278DBB2C7
:100AA000934200D9E6E0A14662004E4BD35A4E492C
:100AB000525A5A40102300210120104201D0013126
:100AC000C9B25208013BDBB2002BF6D1404B1B7878
:100AD000002B06D0454B1A680123484683401A4232
:100AE00001D101293AD92E4BFE221A70F63A5A70DA
:100AF0009E7000229446DA7049462031364A92466A
:100B0000525CD2B20192501CC0B2524650546A4656
:100B100012791A71A2225A7162469A711022DA7100
:100B200031494A465000425AD2B21A72425A120A07
:100B30005A72FFF70BFC1E4B1870284B1B78002BCA
:100B400009D02A490A6801234846834013430B60B1
:100B50000022234B1A80FFF795FB8BE04B465B008E
:100B6000204A9A5A20495B5A5A4000D182E0944662
:100B7000D30712D4012101239A46019410000200E8
:100B80000A415446144233D10133DBB20131102BF8
:100B9000F5D103936246019C2DE0002303932AE0E4
:100BA000BC01002034060020B8010020CD00002048
:100BB000B10100203E030020A50400207C0000209D
:100BC000B0010020990100207C0600205401002083
:100BD0003006002004020020940200202B06002092
:100BE00000020020D00000206403002088000020C4
:100BF00003936246019CFE208D4B1870F9385870A3
:100C00009E700020D870484620308A4B9C460300D6
:100C10006146085CC1B2019101316846C172C17A76
:100C20008A4661465046C854814B69460979197114
:100C30004B4659008048095A0A40511E8A41A12159
:100C40008A1A7B494A716B461B7B8B71FFF77EFBCF
:100C50007A4B18707A4B1B78002B09D079490A68B7
:100C600001234846834013430B600022764B1A80D1
:100C7000FFF708FB754B9B78754A1278DBB29342FD
:100C800000D9BDE0A1466200724BD35A7249525A54
:100C90005A40102300210120104201D00131C9B275
:100CA0005208013BDBB2002BF6D16C4B1B78002BBA
:100CB00006D06B4B1A680123484683401A4201D183
:100CC00001293AD95A4BFE221A70F63A5A709D7091
:100CD00000229446DA7049464031564A9246525CA8
:100CE000D2B20192501CC0B2524650546A46127998
:100CF0001A71A2225A7162469A711022DA7156490B
:100D00004A465000425AD2B21A72425A120A5A72D3
:100D1000FFF71CFB494B1870494B1B78002B09D07F
:100D20004F490A6801234846834013430B60002261
:100D3000454B1A80FFF7A6FA62E04B465B00454A36
:100D40009A5A45495B5A5A405AD09446D30712D40E
:100D5000012101239A460194100002000A415446E1
:100D600014420BD10133DBB20131102BF5D10393C7
:100D70006246019C05E00023039302E00393624670
:100D8000019CFE202A4B1870F93858709D70002085
:100D9000D87048464030274B9C4603006146085CAB
:100DA000C1B2019101316846C172C17A8A46614679
:100DB0005046C8541E4B6946097919714B46590073
:100DC0002548095A0A40511E8A41A1218A1A184908
:100DD0004A716B461B7B8B71FFF7B8FA174B187083
:100DE000174B1B78002B09D01D490A680123484680
:100DF000834013430B600022134B1A80FFF742FA23
:100E00000134E4B2124B1B78DBB20135EDB201368E
:100E1000F6B20137FFB2A34200D97BE50022114BA5
:100E20001A7005B03CBC90469946A246AB46F0BD50
:100E3000BC0100209402002064030020B1010020C6
:100E40002B0600208800002000020020B8010020AE
:100E500099010020080200203406002030060020FE
:100E60009C0100201001002070B50400FFF78CF9F0
:100E70002D4A13780133DBB213701378002B03D1A2
:100E800013780133DBB213702849FE230B70F23B59
:100E90004B7000238B7026480378DBB25A1CD2B209
:100EA0000270CB70204B1B78DBB24B71651CEDB22E
:100EB0008D71204B620010198000C05CC87112193E
:100EC00092009B185A780A729A784A721A798A7232
:100ED0005A79CA729A790A73DA794A739B7ADB076C
:100EE00002D58D220A710AE08C22104B1A71630020
:100EF0001B199B000F4AD31800229A725A60630094
:100F00001C19A4000B4B1C19A37A04229343A3724F
:100F1000FFF71CFA084B1870FFF7B4F9074B1D7068
:100F20008022074B1A7070BD2E060020BC010020E5
:100F3000BB010020A8040020B10100202D060020E4
:100F400028060020F0B55F4656464D464446F0B4AC
:100F500089B0E14B1B78DBB2E04AD35CDBB2FE2BFD
:100F600001D001F01BFEDC4A13780133DBB21370B1
:100F700001F014FE5A1CD1B22278D318DBB2C25C45
:100F8000D2B2FE2A02D00B1EF4D101E0002906D114
:100F90000023D14A1370D24A137001F09FFECE4A4B
:100FA0001370CD4A13780133DBB213701378DBB2C0
:100FB000CA49CB5C0233DFB21478E419C84B1E78FF
:100FC0001B781278DBB2934201D20136FF36C54B53
:100FD0001B78002B1FD1C04B1B78F31AC02B38DDB8
:100FE0000125C04B1D70C04BFE221A7000229A7062
:100FF00004325A70BD480278D2B2511CC9B2017095
:10100000DA708E221A715D71FFF7A0F9B84B187073
:10101000FFF738F91DE0B04B1B78F31A3F2B18DCB3
:101020000025B04B1D70B04BFE221A709D70FA3A2D
:101030005A70AE480278D2B2511CC9B20170DA704F
:101040008E221A715D71FFF781F9A94B1870FFF7B5
:1010500019F9FF232340A14AD35CDBB2FE2B57D002
:10106000A64201D801F03AFE00239B48FF229B498B
:1010700080468C4689468346019604E0019DA54240
:1010800001D801F02BFEBB420ED2019E0478E41879
:1010900014400C5DE4B2FD2C01D10137FFB20133E5
:1010A000DBB29F42F2D8019644462478BDB2029545
:1010B0003C1916002640B24666465546755D002D21
:1010C0000BD1013CA4B215002540AA46834D5646DB
:1010D000AD5D002D01D101F001FE14404D462C5DA7
:1010E000E4B2FE2C14D05C462478013C029DAA4652
:1010F00054441440794D2C5D01373F19FFB25C46D2
:101100002478E41916002640AD5DEDB2FE2DB5D170
:10111000714B1B78013BDBB20021704AD154002F88
:1011200055D0002301936C4A94466C4A934660461E
:101130001600704D704A9146A846CA46624612781B
:10114000D2B259468A5CD2B2FD2A12D16A4A1278CA
:10115000002A0ED10121684A1170013BDBB25E4CBE
:101160002278D2B2511CC9B2217000245B498C5440
:1011700028E01C000278D2B2B25CD2B2EA54027803
:10118000D2B2511CC9B201700021B154EA5CD2B292
:10119000FE2A06D1019ABA1A013A934201DA01F005
:1011A0009DFD4A461278002A0CD04246115DF0227D
:1011B0000A4341460A55002251460A70019A0132FB
:1011C000D2B201920133DBB29F42B7D801E00023D3
:1011D0000193414A137801981B1ADBB213701378FC
:1011E000DBB2591CC9B2117000213C4AD154831C96
:1011F000DBB2069300230593404B683307933D4BC6
:101200005B78002B01D000F03AFD374BFE221A70BC
:1012100000229A70374BDB78DBB2312B01D900F01A
:101220000DFD9B00364AD3589F46324B9A790023D6
:10123000002A01D000F022FC00F02BFC2B490023F7
:101240000B70294B05225A700A78D2B2501CC0B2DA
:101250000870DA7081221A717D325A714F3A9A7190
:10126000FFF774F8224B187000F0E8FC0023254AC1
:101270001370254A137000F0E1FCFEF785FF234947
:101280000A7848788B782249097882189B18CB18FD
:10129000DBB21A4A1370144904224A70134C2278A4
:1012A000D2B2501CC0B22070CA7088220A71194A8A
:1012B00011780022002900D01A000B4B5A71FFF759
:1012C00045F80B4B18700D4A002353709370124A67
:1012D000137000F0B3FCC04675060020A403002084
:1012E000840000203F030020BC010020BB0100203F
:1012F000B1010020540200202C0600200C00002028
:101300005C4B00002D06002028060020B8010020BC
:10131000A4040020410300204A030020E54B9A78F2
:101320001B78934200D8E4E0E34B1B78002B04D1F8
:10133000E1490B780133DBB20B70002A00D1B1E038
:10134000DC4B5B781F2B29D85A00D2189200DB495E
:101350008A18927AD20719D501F068FC581CC0B2DD
:101360005900C9188900D54CA4466144897AC90737
:101370000FD5D0494B705900CA189200A218917A23
:101380000420814391721F2B5BD907E00133DBB24C
:1013900000E00300202BE1D1C64A5370C84B1B78F4
:1013A000C84A1278DBB22020934204D8C44B187884
:1013B00040231B1AD8B2C34B1A78D2B2C0490B785B
:1013C0004978CB189A4206DBBD4A13785078C0188A
:1013D00060231B1AD8B2BC490C234B70BB4C23783A
:1013E000DBB25A1CD2B22270CB7089230B71B24B84
:1013F0001B78DBB24B71B34D2B781B18DBB28B71B2
:101400004023CB7100230B723E334B72B04C2368E8
:101410001B0E8B728B7A0133DBB28B7222682B78B6
:10142000DBB25E1CF6B22E70120C9B18C318DBB236
:10143000CB7223681B0ADBB20B732368DBB24B73DE
:1014400065E0A1490C234B70A0480378DBB25A1C1D
:10145000D2B20270CB7089230B71974B1B78DBB231
:101460004B71944B98465B78581CC0B28871934C72
:101470005E00F2189200125DCA71F2189200A21872
:1014800055780D7295784D7215798D725579CD72AA
:1014900092790A73F3189B00E318DB794B73434688
:1014A000587034E088490C234B7088480378DBB2CD
:1014B0005A1CD2B20270CB7089230B717E4B1B7801
:1014C000DBB24B7100238B718022CA710B723E33E9
:1014D0004B727F4A13681B0E8B7213681B0CDBB2B6
:1014E000CB7213681B0ADBB20B731368DBB24B734E
:1014F0000DE0754B04225A7074480278D2B2511C28
:10150000C9B20170DA708B221A7174325A71FEF707
:101510001DFF704B1870674A9378013393708DE309
:10152000694B05225A7069480278D2B2511CC9B27F
:101530000170DA7083221A717C3A5A7100229A7112
:10154000FEF704FF634B187078E35F490A234B7082
:101550005E480378DBB25A1CD2B20270CB7084238F
:101560000B71043B4B7100238B713E33CB71584A96
:1015700013681B0E0B7213681B0CDBB24B721368E3
:101580001B0ADBB28B721368DBB2CB72FEF7DEFE96
:10159000504B187052E34C4B06225A704B4802785D
:1015A000D2B2511CC9B20170DA7085221A71843A24
:1015B000DA7102329A7100225A71FEF7C7FE454B6A
:1015C00018703BE3404B04225A7040480278D2B274
:1015D000511CC9B20170DA7082221A713E4A127926
:1015E000D2B25A71FEF7B2FE3A4B187026E30022CF
:1015F0003A4B1A70E8E20123394A1370374A1370E4
:10160000384A1370E0E2304B04225A702F480278B7
:10161000D2B2511CC9B20170DA7092221A71903A9A
:101620005A710022234BDA70FEF790FE294B187096
:1016300004E3294B1B79DBB2FC2B05D0FD2B07D132
:1016400000221C4BDA700AE001221A4BDA701BE010
:10165000184BDB78002B02D0012B45D114E01A4B3C
:1016600005225A7019480278D2B2511CC9B20170D1
:10167000DA7090221A716D325A71F53A9A71FEF74A
:1016800065FE144B187043E00F4B05225A700F484B
:101690000278D2B2511CC9B20170DA7090221A716C
:1016A0006C325A71E43A9A71FEF750FE094B187089
:1016B0002EE0C0460C0000202E060020A8040020CA
:1016C000B80100204A030020BC010020BB0100201B
:1016D00078000020B101002054020020A504002061
:1016E000B001002010010020D94B04225A70D948C3
:1016F0000278D2B2511CC9B20170DA7091221A710B
:10170000D54A1279D2B25A71FEF720FED34B187027
:10171000D34AD3780133D37090E2D24B1B78002B9D
:1017200005D00023CF4A1370CF4A136002E0012294
:10173000CC4B1A70C64A04235370C6480378DBB2F8
:10174000591CC9B20170D37087231371C54B1B7824
:10175000591E8B41DBB25371FEF7F8FDBF4B187079
:101760006CE2BB4B04225A70BA480278D2B2511CC8
:10177000C9B20170DA708A221A710A3A5A71FEF7F8
:10178000E5FDB64B187059E2B84B1B78002B00D121
:1017900054E2B14B1C79E4B2092C04D90022B34BBA
:1017A0001A7001F09BFA611DAB4B5D5CEDB2092D27
:1017B00004D90022AD4B1A7001F090FA631DEB18AA
:1017C000DBB2A34A5370A34E3378DBB2581CC0B2CD
:1017D0003070D370932313719F4B1B79DBB253711D
:1017E000002C12D0621ED2B2063205239A488446DB
:1017F000974E8846581C6146CB5CDBB233540300DD
:101800008242F7D14146230000E023000633924A8A
:10181000525CD2B28E49CA54002D01D101F0D3F9E5
:10182000A31D691EC9B2E21D89188B4E88485A1C37
:10183000F35CDBB2835413009142F8D1FEF786FDCE
:10184000864B1870844B5B79303BDBB2012C0ED990
:1018500006200121804E9A009B185B00325C303AD2
:101860009B18DBB20131C9B201308C42F3D8A21D02
:1018700079498A5C303AD2B2012D0FD9E01D083483
:10188000023DEDB264190D00910052185200295C1E
:1018900030395218D2B201308442F5D1032B00D92D
:1018A000CCE1111C322A00D93221013B704AD154BB
:1018B0000122704B1A70C1E16C4B1B78002B00D1D8
:1018C000BCE1654B1C79E4B2092C04D90022674BBA
:1018D0001A7001F003FA604B5B79303BDBB2012CEC
:1018E0000ED9A01EC0B2073006215B4D9A009B188E
:1018F0005B006A5C303A9B18DBB201318842F5D15B
:1019000022000832D2B252484270524D2A78D2B2E6
:10191000511CC9B22970C270932202714E4A1279C9
:10192000D2B24271002C0CD0611EC9B20631052220
:10193000494E0500501CB25CD2B22A54021E8A42A3
:10194000F8D1A21D032042498854032B21D8E21D5F
:101950000E003021B154013B454AD05CC0B2343155
:1019600003F0B8F8CDB208239846A0440A21280015
:1019700003F02AF803003033DBB24246B354093493
:101980000A21280003F0A6F80B003033DBB23355F0
:1019900009E0E21D2E4B32219954210008313522F5
:1019A0005A5409341A55FEF7D1FC2C4B187045E1F6
:1019B00000202E4B1870264B04225A70254C22789A
:1019C000D2B2511CC9B22170DA7094221A715871C6
:1019D000FEF7BCFC214B187030E11F4BDA79D2B214
:1019E000254B1B681B0E9A4200D027E11A4B1A7A2E
:1019F000D2B2214B1B681B021B0E9A4200D01DE184
:101A0000154B5A7AD2B21C4B1B681B041B0E9A4210
:101A100000D013E1104B9B7ADBB2174A1268D2B2A6
:101A20009A4200D00AE10120104B1870084B0422A2
:101A30005A70084C2278D2B2511CC9B22170DA70A7
:101A400094221A715871FEF781FC044B1870F5E06E
:101A5000BC010020BB01002054020020B101002085
:101A60000C0000204B030020944200502A06002066
:101A7000B8010020A604002078000020DF49E048DB
:101A8000DA1D8A5CC2540133DBB28A79D2B29A423F
:101A9000F6D80021DA4AD154D84B01225A71D949DB
:101AA0000A705B79002B04D137E0D44B5B79002BB3
:101AB00033D0D34B1B78002B01D101F091F8D24ADF
:101AC00001231178002906D00133DBB20132182B33
:101AD000F7D101F0B6F8991DC9B2CC4A5170CC4C7F
:101AE0002178C9B2481CC0B22070D1709521117103
:101AF0000021517101319171D371002B29D0591EF0
:101B0000C9B209310823BE4CC0481A00083AA25C89
:101B1000C25401338B42F8D11BE0BC490C234B70FB
:101B2000BB480378DBB25A1CD2B20270CB7095234B
:101B30000B7100234B718B710633CB7154330B72D5
:101B40000B334B7210338B72023BCB72533B0B73D4
:101B50004B73FEF7FBFBAF4B18706FE0AB490523EF
:101B60004B70AB480378DBB25A1CD2B20270CB7018
:101B700086230B71A84B1B78DBB24B7100238B7152
:101B8000FEF7E4FBA34B187058E00023A04A137043
:101B9000A24A1370A24A1370A24A1360A24A137099
:101BA000A24A13700022A24C012053009B189B00F4
:101BB000E318997A814399720132202AF5D103E022
:101BC0008E4B1B79002B39D19A4B00221A70781E4C
:101BD000C2B25A7089490A78D2B29A704A78D2B29F
:101BE000DA7002280CDD022202230D00914C911CB8
:101BF000AA5CD2B262540133DBB21A1E8242F6DB17
:101C000000228D4B1A708D488D4A01211D001C0049
:101C10000FE09368194206D093680B4393602B78CA
:101C20000133DBB22B702378DBB2142B01D900F027
:101C300050FF0378002BECD100F04BFF6F4B1B786B
:101C4000069A944663449F4201DC00F08FFF6B4B81
:101C500018780130C0B23F1AFFB2002F01D1FFF750
:101C6000CEFA7C1EE4B2013400236449C2188A5CB7
:101C7000D2B2CA5401339C42F8D1FFF7C0FA5F4B8D
:101C80005B78DBB21F2B01D800F0B4FE5B4B9B7876
:101C9000002B01D000F0AEFE584B5B78DBB25F2B1F
:101CA00005D9564B5B78203BDBB298460FE0534B8F
:101CB0005B78DBB23F2B05D9504B5B78203BDBB226
:101CC000984604E04D4B5B78203BDBB298464F4B87
:101CD000FE221A7049494A78D2B29A700022DA700C
:101CE0000B79DBB2252B01D900F064FE9B00554A2D
:101CF000D3589F465449002342468B54434B0622F7
:101D00005A7042468A5CD2B2501CC0B24446085552
:101D10001A7181225A717D329A714F3ADA71FEF747
:101D200015FB3C4B187000F045FE384B06225A70EC
:101D300045484246825CD2B2511CC9B24446015564
:101D40001A7183225A717C3A9A710022DA71FEF775
:101D5000FDFA304B187000F02DFE00223B4B1A703C
:101D600000F028FE0122394B1A7000F023FE274AAA
:101D70000B23537034484346C35CDBB2591CC9B2D1
:101D800044460155137184235371443B93710023DE
:101D9000D3713E3313722E490B681B0E53720B68BE
:101DA000164840781B0C1B1A4433DBB293720B6845
:101DB0001B0ADBB2D3720B68DBB21373FEF7C6FAF1
:101DC000144B187000F0F6FD104907234B701E48A5
:101DD0004346C35CDBB25A1CD2B2444602550B7177
:101DE00085234B7100238B710333CB71023B0B7244
:101DF000FEF7ACFA074B187000F0DCFD540200202F
:101E00004C030020780600204D030020BC01002078
:101E1000BB010020B1010020CC000020750600208D
:101E2000840000209401002048030020410300208A
:101E3000A8040020FC020020740600209801002065
:101E400020000140244C000094020020B00100203A
:101E500078000020B34905234B70B3484346C35C68
:101E6000DBB25A1CD2B2444602550B7182234B712D
:101E7000AE4B5B79DBB28B71FEF768FAAC4B187036
:101E800000F098FDAB4B1B78002B05D00023A94A2E
:101E90001370A94A136002E00122A64B1A70A149EF
:101EA00005234B70A0484346C35CDBB25A1CD2B238
:101EB000444602550B7187234B719E4B1B785A1E6B
:101EC0009341DBB28B71FEF741FA994B187000F029
:101ED00071FD944B05225A7093484246825CD2B2FF
:101EE000511CC9B2444601551A718A225A714A3AA4
:101EF0009A71FEF72BFA8E4B187000F05BFD8B4B3E
:101F0000DB79DBB2102B02D91022884BDA71874BB8
:101F1000DB79002B0DD00023844988481A00083251
:101F20008A5CC2540133DBB2CA79D2B29A42F5D884
:101F300000E000230021814AD15401227B4B9A7199
:101F40001F254545AD416D426B02029343463F2B31
:101F500002D98023DB000293A022D20580235B00FC
:101F6000592616248820D650D450D050D158002954
:101F7000F9D0734B1A6801210A431A602222DA60F1
:101F8000FD2252025A601961BFF36F8F1A00136964
:101F9000002BFCD1FD22520202990B00FA204002D4
:101FA0008446634404930B0066498C4663449B4615
:101FB000634B0024012021218A46FE2149028C46E0
:101FC000B9465E4604990391029FB118DC605960DE
:101FD0009C601861BFF36F8F19690029FCD1996863
:101FE0005546DD605A6099601861BFF36F8F1969BB
:101FF0000029FCD104326245E4D13E004F46504BEB
:102000002222DA60039A5A6001221A61BFF36F8FAD
:102010001A69002AFCD149480178090643781B0453
:10202000C91883781B02CB18C1785B1802931F254F
:1020300043461D40424B0121FA2040028146B144F3
:102040003E4884464846B946070094B22409A54252
:1020500000D07FE0BC182120D8605C6002989860B6
:102060001961BFF36F8F1C69002CFCD133480479D0
:10207000200683463148447924045C44A24684798E
:1020800024025444C079824654442F488246B244C4
:1020900092442120D860504658609C601961BFF37B
:1020A0006F8F1C69002CFCD12448047A20068346DB
:1020B0002248447A24045C44A246847A240254448C
:1020C000C07A8246544421488246B2449244212038
:1020D000D860504658609C601961BFF36F8F1C69CF
:1020E000002CFCD16046047B200683466046447B7E
:1020F00024045C44A246847B24025444C07B824670
:10210000544413488246B24492442120D860504639
:1021100058609C601961BFF36F8F1C69002CFCD163
:102120008AE0C046BC010020940200205402002036
:10213000B10100204B03002094420050A001002078
:1021400000C0005000FAFFFF04F4010008F4010091
:102150000CF401000020D860FD24640214195C60B6
:1021600098601961BFF36F8F1C69002CFCD19C68CB
:10217000A246BC182120D8605C6050469860196166
:10218000BFF36F8F1C69002CFCD10020D860D748AA
:1021900014185C60002098601961BFF36F8F1C6990
:1021A000002CFCD198688246D1483418A41821200C
:1021B000D8605C60504698601961BFF36F8F1C69EE
:1021C000002CFCD10020D860CA4814185C600020A4
:1021D00098601961BFF36F8F1C69002CFCD198685F
:1021E0008246C5483418A4182120D8605C60504647
:1021F00098601961BFF36F8F1C69002CFCD100201F
:10220000D860BE4814185C60002098601961BFF364
:102210006F8F1C69002CFCD198688246B84834182E
:10222000A4182120D8605C60504698601961BFF303
:102230006F8F1C69002CFCD110328024A400A242B4
:1022400000D002E74F46AF4A136801218B43136069
:10225000002180235B00A022D205D150AA4B9B799C
:10226000002B7ED0A022D20580235B0059251624A6
:102270008820D550D450D050D1580029F9D0A14A47
:10228000116801230B4313604546FA24640144445A
:1022900024019E4810239846A044010000239C4638
:1022A000013399466346D360546093604B46136193
:1022B000BFF36F8F1369002BFCD193681E0E0E7055
:1022C0001E0C4E701E0A8E70CB70043404314445CF
:1022D000E8D18C4A136801218B43136000218023CD
:1022E0005B00A022D205D150884B1B78FF2B05D173
:1022F000864B20221A7000225A7007E0002B05D16D
:1023000000F081FC4378002B02D108E00121F9E7BD
:102310000131C9B201301029F4D100F0CBFCCB1D42
:10232000DBB27B4843707B4C635DDBB25A1CD2B29C
:102330006255037195234371002383710133C37187
:10234000017200294AD00139C9B20A3109236F4C00
:102350006F481A00093AA25CC25401339942F8D17D
:102360003CE06B4C152363706A494346CB5CDBB29F
:102370005A1CD2B240460A5423719523637100233C
:10238000A371E3710E332372653363723B3BA37217
:10239000E3720B3B2373203363732233A3730B3B32
:1023A000E37311332374093B63744C3BA3744309F7
:1023B0003133E3742E2323751F2505400A2128009D
:1023C00002F002FB03003033DBB263750A21280000
:1023D00002F080FB0B003133DBB2A375FDF7B6FFD3
:1023E0004D4B1870E6E24A4B05225A704948424666
:1023F000825CD2B2511CC9B2444601551A71922274
:102400005A718C3A9A71454B0433002207991A701D
:1024100001339942FBD1FDF799FF3F4B1870C9E298
:10242000394B5B78DBB23F2B04D8374B5B78203BD2
:10243000DBB215E0344B5B78DBB25F2B07D8324B55
:102440005B78374A1278D318403BDBB208E02E4B5A
:102450005A7833490B7849789B18603BCB18DBB22C
:10246000294A5279D2B2022A16D004D8002A09D0B9
:10247000012A0CD023E0FC2A1DD0FD2A16D0032A05
:102480001DD10EE0254AD31800221A7117E0234A05
:10249000D31801221A7112E0204AD31802221A71AD
:1024A0000DE01E4AD31803221A7108E01B4AD31804
:1024B00004221A7103E0194AD31805221A71124B2B
:1024C0005B78DBB23F2B04D80F4B5B78203BDBB251
:1024D00031E00D4B5B78DBB25F2B23D80A4B5B7886
:1024E0000F4A1278D318403BDBB224E004FA010013
:1024F00004F4010008FA010008F401000CFA0100DC
:102500000CF4010000C0005054020020A001002083
:10251000BC01002094020020B10100200C0000202A
:10252000B8010020E44B5A78E4490B7849789B18AD
:10253000603BCB18DBB21900E14AD2181279052AA8
:1025400000D9ACE09200DF4B9B589F46DE48062343
:102550004370DE4C4346E35CDBB25A1CD2B24546C4
:102560006255037190234371002383711033C3714B
:10257000D34B5B1801221A71FDF7E8FED44B18709B
:1025800018E2D14806234370D04C4346E35CDBB2EB
:102590005A1CD2B2454662550371902343718F3B5A
:1025A0008371CC4B1A78531E9A41D2B2C271C44B7C
:1025B0005B1802221A71FDF7C9FEC54B1870F9E1CC
:1025C000C14806234370C14C4346E35CDBB25A1C4E
:1025D000D2B2454662550371902343718E3B83719D
:1025E000013BC371B64B5B1803221A71FDF7AEFEB7
:1025F000B74B1870DEE1B44806234370B34C434632
:10260000E35CDBB25A1CD2B245466255037190239B
:1026100043718D3B8371B04B1A78531E9A41D2B2ED
:10262000C271A74B5B1804221A71FDF78FFEA84BED
:102630001870BFE1A44806234370A44C4346E35CF2
:10264000DBB25A1CD2B245466255037190234371E6
:102650006D338371F53BC371994B5B1805221A7179
:10266000FDF774FE9A4B1870A4E197480624447055
:10267000964D4346EB5CDBB25A1CD2B24646AA5595
:102680000371902343716C338371EC3BC3718C4BAA
:102690005B181C71FDF75AFE8D4B18708AE18A4C4D
:1026A00005216170894D4146695CC9B2481CC0B2C0
:1026B0004646A8552171912161717F494979C9B276
:1026C000A1717F49CB1801321A71FDF73FFE804B93
:1026D00018706FE1784B5B79DBB2012B1BD0002BBC
:1026E00002D0032B3FD067E0774B05225A70774822
:1026F0004246825CD2B2511CC9B2444601551A719D
:1027000090225A7100229A711032DA71FDF71EFE82
:102710006F4B18704EE1684B9B79002B03D0012260
:102720006C4B1A7002E000226A4B1A70664906234D
:102730004B7066484346C35CDBB25A1CD2B2444677
:1027400002550B7190234B7101248C71614B1B78E6
:102750005A1E9341DBB2CB71FDF7F8FD5C4B18704C
:102760005E4B1C7026E1544B9B79002B03D0012259
:10277000594B1A7002E00022574B1A705249062337
:102780004B7052484346C35CDBB25A1CD2B244463B
:1027900002550B7190234B718D3B8B714E4B1B7807
:1027A0005A1E9341DBB2CB71FDF7D0FD484B187038
:1027B00001224A4B1A70FDE0434905234B70434800
:1027C0004346C35CDBB25A1CD2B2444602550B717D
:1027D00091234B71384B5B79DBB28B71FDF7B6FD02
:1027E0003B4B1870E6E0344948798B79DB08C00828
:1027F000181AC0B2831DDBB2334A5370334D4346BF
:10280000EB5CDBB25C1CE4B24646AC551371A22310
:1028100053714B79DBB29371C300DBB2D3710028E3
:1028200075D005000935EDB209230E001A00093AEA
:10283000D1B25A1ED4B27278D2B25F2A15D9CA0761
:1028400009D51D4A5278603A52002549525A120A57
:102850001D490A5553E0184A5278603A52002049FF
:10286000525AD2B218490A5549E0134A5278D2B2A4
:102870003F2A15D9CA0709D50F4A5278403A520063
:102880001849525A120A10490A5538E00A4A527831
:10289000403A52001349525AD2B20B490A552EE01F
:1028A000CA0723D5044A5278203A52000E49525A98
:1028B000120A05490A5522E054020020B8010020FE
:1028C0000C000020BC4C0000BC0100209402002041
:1028D000B10100207C0000202B060020A60400206F
:1028E00008020020D00000207C060020DF4A527839
:1028F000203A5200DE49525AD2B2DE490A5501331B
:10290000DBB2AB4292D10830C3B2059301E0082399
:1029100005930023D84A1360D84A1360D84A13603D
:10292000FDF714FDD74B187044E0D24B07225A70C4
:10293000D5484246825CD2B2511CC9B244460155C8
:102940001A71A9225A7100229A71DA711A72FDF76E
:10295000FDFCCC4B18702DE0C44B5B78DBB21A0049
:10296000203AD2B21F2A09D8C348036801219140F6
:102970008B4303600022C54B1A7018E03F2A0BD826
:10298000BE480268403BDBB2012199408A430260A5
:102990000022BE4B1A700AE0B9480268603BDBB205
:1029A000012199408A4302600022B84B1A7000222C
:1029B000B44B1A70AD4B1B78069A944663449F4201
:1029C00000DCD3E0A94B18780130C0B23F1AFFB247
:1029D000002F01D1FEF713FC7C1EE4B2013400236A
:1029E000A249C2188A5CD2B2CA540133A342F8D1B8
:1029F000FEF705FCA64A00231370019BFB1ADBB20D
:102A000053709A490B78DBB293704B78DBB2D3707A
:102A1000022F0FD9FC1EE4B2033402230E00110072
:102A20000025981CF25CD2B20A545A1D8D54013311
:102A30009C42F6D1964B9B780222069BFB1A944847
:102A40000EE0815C01315218D2B2111F7C2907D9E6
:102A500001238F490022CA5401333C2BFBD13DE1B5
:102A60009A42EEDB023AD2B2894B5A700022894B6D
:102A70001A70894D894A0124180019000DE09368E5
:102A80001C4206D093682343936003780133DBB282
:102A900003700B78DBB2142B02D82B78002BEED10D
:102AA00000227C4B1A7018007C4A01211C0009E0AE
:102AB0009368194206D093680B43936023780133DF
:102AC000DBB223700378DBB2012BF1D90022714B0A
:102AD0001A706F4B5C78E4B23F2C47D87049802263
:102AE00012048B691342FCD10020FDF7F9FB6C4BFB
:102AF000D96810220A43DA60D96820220A43DA60D2
:102B0000D96808220A43DA60631C99460127012626
:102B1000634C80252D045E4B984600239A46A3699A
:102B20002B42FCD14346DB5DDBB223604346D85DDC
:102B3000059B5840C0B2FDF74BFB059043465246FB
:102B4000DA550136F6B2371E4F45E8DD544980228A
:102B500012048B691342FCD1514B059A1A60012370
:102B60004B490022CA5401333C2BFBD1454B1B7807
:102B7000002B00D1B2E0FDF785FBAFE0494B1B789D
:102B80000133DBB2484AD25CD2B2FE2A01D1FEF751
:102B900006FA0223434C4448FEF7ECF9414A137805
:102BA000013BDBB213701378DBB23F4AD35CDBB27C
:102BB000FE2BE3D1FEF7F5F906342C4A125D303ACC
:102BC000D2B2FEF76BFEFDF7C1FB2E4B1870274B00
:102BD0005B79303BDBB2012C01D9FEF739FEEBE724
:102BE000244B06225A7031480278D2B2511CC9B225
:102BF0000170DA7095221A7100225A7101219971BF
:102C0000DA71FEF7A6FF1B4B07225A701E48425D81
:102C1000D2B2511CC9B241551A7195225A71002283
:102C20009A710121D9711A72FFF7D8FB5A00D31893
:102C30009B001F4AD3189A7A04218A439A72FEF79E
:102C400000FC0C481E224270184C2278D2B2511C53
:102C5000C9B22170C2709522027100224271013204
:102C600082711732C271FEF74AFFC046540200203B
:102C70007C060020BC010020040200208800002007
:102C80009C010020B1010020940200207706002062
:102C9000FC02002074060020980100202000014062
:102CA0000000154075060020A4030020BB01002091
:102CB000A80400200D48172343700D4C635DDBB260
:102CC0005A1CD2B26255037195234371002383715C
:102CD0000133C3710F330372FFF735FB09B03CBCFE
:102CE00090469946A246AB46F0BDC046BC010020C6
:102CF00094020020F0B55F4656464D464446F0B477
:102D000085B08F4D8F4B2B608F4C904B236090483C
:102D1000904A026090490B60904A914B13600023E7
:102D2000AB60A360836080338B60703B9360A022B4
:102D3000D205F033592416208821D450D050D150D8
:102D4000D558002DF9D0874A116801230B43136031
:102D5000854B1100012202E0013B002B02D0C86824
:102D60000242F9D07F4B00221A611A6A802149027F
:102D70000A431A627D4A1A627B4B7A49042202E0B6
:102D8000013B002B02D0C8680242F9D0754B0222E9
:102D90001A61774A9A6000225A6101F077FD012397
:102DA000744A1360744A11680B431360734AF92123
:102DB0004902714B00240126714DDC6059609C6012
:102DC0001E61BFF36F8F18690028FCD19868070E49
:102DD0001770070C5770070A9770D07004310432CF
:102DE000A942EAD1654B1B78FF2B04D1634B20220B
:102DF0001A7000225A70604B0022DA6061495960F3
:102E00009A6001321A61BFF36F8F1A69002AFCD1F0
:102E1000594B9A685C490A600A681204120C0A60ED
:102E20000022DA60F821490259609A6001321A6181
:102E3000BFF36F8F1A69002AFCD14F4B9B68D9B240
:102E4000524A1170DA0503D50121514A117002E08E
:102E500000214F4A11709B0503D501224D4B1A707A
:102E600002E000224B4B1A70434B0022DA604A49C1
:102E700059609A6001321A61BFF36F8F1A69002A94
:102E8000FCD13D4A936811680120814311603E499D
:102E90000A6890200006844662440A60D9B23F4A1C
:102EA0001170190AC9B251701B0CDBB29370137800
:102EB000DBB2202B02D90122384B1A70374B5B78DA
:102EC000DBB2202B02D90122344B5A70334B9B7852
:102ED000DBB2202B02D90122304B9A702F4A137893
:102EE0005278DBB2934205D92C4B1B78DBB2274AD0
:102EF000137004E0294B5B78DBB2244A1370274B34
:102F00009B78224A1278DBB2934204D9234B9B78F8
:102F1000DBB21E4A13700322A023DB05DA63204BC9
:102F20001B68002B42D1023A1E4B1A70962080017A
:102F3000FDF702F9C0239B0518431B4B58623EE086
:102F400000400050F7FF000040400050FFFF00002D
:102F50008040005015150000C04000500041005056
:102F600015FF00000002005091D00300174200003E
:102F7000080003009442005000C000504C030020A1
:102F800018F20100FC0F10007800002099010020C9
:102F90007C0000202B06002004F00100B801002076
:102FA0007C420050F802002000000540E120400271
:102FB000FDF7C2F8C0239B051843DB4B5862DA4B80
:102FC00003229046DA605A6801273A435A60D74C88
:102FD000C326B600A359FF2293431A00402313438C
:102FE000A35180235B012360A025ED05C0231B01B5
:102FF0006B63C0239B002B63CD48FDF79DF8C02376
:103000009B051843CB4B58620B22DA6042461A6389
:103010008022D200DA629A68F0218A439A60002105
:1030200019615A6817435F6080239B012360A2598E
:10303000C14B1A40A251C14A11608020C0041060E7
:10304000BF481060BF485060C2229200A0580340A1
:10305000C02000020343A35080235B00E950A73B3C
:103060009B46B94B1B78002B5ED0A022D205802353
:103070005B00162488205946D150D450D050D158E6
:103080000029F8D0B14B1A6801210A431A602222A4
:10309000DA60F82252025A601961BFF36F8F1A008A
:1030A0001369002BFCD1AA4B1B78DBB2A94A12781A
:1030B000002A02D0802252001343A74A1278002A25
:1030C00002D0802292001343A04A2121D160F8212E
:1030D00049025160936001231361BFF36F8F13693D
:1030E000002BFCD19D4A1178537892781B02CB18A3
:1030F00012049B18954A2121D1609949516093602F
:1031000001231361BFF36F8F1369002BFCD18F4A2A
:10311000136801218B431360002380225200A021F9
:10312000C9058B50884A13708E4B1B78002B56D0E4
:10313000A022D20580235B00162488205946D15056
:10314000D450D050D1580029F8D0804B1A680121B2
:103150000A431A602222DA60F82252025A60196188
:10316000BFF36F8F1A001369002BFCD1774B22221B
:10317000DA60F92252025A6001221A61BFF36F8F9E
:103180001A001369002BFCD17748F92464026F49B7
:1031900021270126754D03781A0643781B04D3189E
:1031A000827812029B18C2789B18CF604C608B60AB
:1031B0000E61BFF36F8F0B69002BFCD10430043418
:1031C000AC42E8D1614A136801218B4313600023AC
:1031D00080225200A021C9058B50624A1370644BB3
:1031E0001B78644A1278DBB2934201D0FDF7AAFE45
:1031F000614B1B78614A1278DBB2934200D133E312
:103200005D4B1B78002B36D1FF33FF335C4AD35A1A
:103210009BB280225200934222D057490B78DBB2F6
:103220005A1CD2B20A705B00554A9B5A9BB280224C
:103230005200934214D0023A0800514D8024640099
:103240000378DBB2591CC9B201705B005B5B9BB2B7
:10325000A34205D0013AD2B2002AF1D101F00EF911
:10326000454B1B785B00464A9B5A9BB2802252001A
:1032700093422ED03BE0404B1B78013B5B00404A21
:103280009B5A9BB2802252009342E9D03A490B7874
:10329000DBB25A1CD2B20A705B00394A9B5A9BB20D
:1032A000802252009342DBD0023A0800344D802441
:1032B00064000378DBB2591CC9B201705B005B5B30
:1032C0009BB2A342CCD0013AD2B2002AF1D101F094
:1032D0000DF9294A2A488021490013780133DBB2CD
:1032E000137013785B001B5A9BB28B42F5D0224BB4
:1032F0001B785B00224A9B5A9BB2002B00D1B3E2A1
:103300001D4B1B785B009A5AD2B2931CDBB2402B48
:103310003CD90023194A13701A4A1370164A1370C5
:10332000194A1370A0E2C0460000054000E100E029
:1033300020A1070000001540FF00FFFF2000014012
:10334000000001685D020000A604002000C00050DB
:10335000990100207C0000202B060020B8010020ED
:1033600004F00100780600204C03002018F2010050
:103370008400002075060020BF080020BD08002042
:10338000BC0600209801002029060020AF490978DA
:10339000C9B2142908D9AE490978C918C9B2490077
:1033A0008024A400AB480C52A9490978C918C9B2B5
:1033B0004900A848095A89B280208000814200D083
:1033C00052E2A34D29780139C9B2A248490000242C
:1033D0000C522978C918C9B249000C52002B01D1EE
:1033E00001F08FF8571CFFB2013700202E00994BD7
:1033F0009846994D3378DBB25A1CD2B232705B00DA
:1034000042469B5ADBB22B552B5D5840C0B2FCF7AD
:10341000DFFE0134A742EDD18D4A13780133DBB2D0
:1034200013708D4B1B79DBB2F02B00D093E1002899
:1034300000D019E28848047A417A827AC37A090274
:10344000611812048A181B06D318844A1360844832
:1034500000210022834C814D4B005B189B00E31838
:103460009B7ADB0732D52B6806689E422ED17E4BB5
:10347000FE221A70F33A5A7000229A707B48027842
:10348000D2B2511CC9B20170DA7086221A71743A34
:103490005A71714A5179C9B299719179C9B2D97188
:1034A000D179C9B21972117AC9B25972517AC9B2B5
:1034B0009972917AC9B2D972D27AD2B21A73FCF7E0
:1034C00045FF6B4B1870FCF7DDFE98E00132D2B27D
:1034D00001310C30202ABFD1624B9B7ADB0701D42B
:1034E00001F01DF81F3A5F49D4B253009B189B00AE
:1034F000CB189B7ADB0701D401F012F80132202AA5
:10350000F2D17CE02000FDF7AFFC63001B199B00AB
:10351000544AD3189B7ADB0709D40CE063001B19CB
:103520009B00504A944663449B7ADB0703D50134E1
:10353000E4B21F2CF2D9202C07D101224D4B1A7076
:103540004D4C4E4A012021000DE00022494B1A70DB
:10355000F6E79368184206D09368034393600B78AC
:103560000133DBB20B702378DBB2042BF1D90022DC
:10357000414B1A70424B5E78F6B2424A80231B04DC
:1035800091691942FCD10020FCF7AAFE3D4BD96895
:1035900010220A43DA60D96820220A43DA60D96827
:1035A00008220A43DA601E603000FCF711FE013683
:1035B000012E18DD02270222324C80252D04304BCB
:1035C0009846A3692B42FCD143469B5CDBB2236047
:1035D00043469B5C5840C0B2FCF7FAFD0137FFB28E
:1035E0003A1EB242EDDD274A80231B04916919423D
:1035F000FCD1244B18600022234B1A6034E1204B8D
:1036000000221A700B21597001399970DA701A7101
:1036100072325A71104A5179C9B299719179C9B20D
:10362000D971D179C9B21972117AC9B25972517A64
:10363000C9B29972917AC9B2D972D27AD2B21A73D6
:103640000D4C0E4A012120002AE0C0462906002028
:10365000BF080020BC060020140100204403002005
:10366000AC040020A8040020BC010020BB01002005
:10367000B1010020B20100207406002020000140AA
:10368000FC0200200000154094420050936819424B
:1036900006D093680B43936003780133DBB2037069
:1036A0002378DBB2132BF1D90022D04B1A70D04B08
:1036B0005F78FFB2CF49802212048B691342FCD19C
:1036C0000020FCF70DFECB4BD96810220A43DA60CC
:1036D000D96820220A43DA60D96808220A43DA60EE
:1036E0001F603800FCF774FD0137012F18DD02263A
:1036F0000222C04C80252D04BD4B9846A3692B4265
:10370000FCD143469B5CDBB2236043469B5C584044
:10371000C0B2FCF75DFD0136F6B2321EBA42EDDDF5
:10372000B449802212048B691342FCD1B14B18605A
:103730000022B14B1A600023B04800215A001152F8
:103740000133402BFAD10023AD4A1370AD4A1370F8
:10375000AD4A137088E000286AD1AC4B1F7801375E
:10376000FBB29A46012400230193FE336A46D373C9
:103770005346019A9E1AF3B29A46A54B6A46D27BEB
:103780001A70631CDBB2A14A155D0135EAB20192E1
:10379000111E402968D89E4842709E4A1278D2B2C3
:1037A00082700A00894602329046032A13DD032202
:1037B000964F03210E1B0025B44646465C1CE4B21E
:1037C000F95CC9B281546344DAB2131DC5542300B5
:1037D000B242F3DB00E01C00FCF7B8FD8E4B187022
:1037E0001B78002B13D000208C4A802109048C4DBB
:1037F0000026894F93690B42FCD12B5CDBB213602E
:103800002E540130C0B23B78DBB29842F2D3002292
:10381000814B1A700132784B1A604F460137BA4516
:1038200022DD00221A607C490A7001321A609FE78B
:10383000774BFE221A70F93A5A7000229A70794832
:103840000278D2B2511CC9B20170DA7086221A71A4
:10385000843A5A716D4AD278D2B29A71FCF776FDE9
:103860006D4B1870FCF70EFD6F4B9B68DB0700D4A7
:103870004AE26D4A916801230B439360614B1B78C8
:10388000002B04D0694A13780133DBB21370684A05
:10389000138801339BB21380664A13780133DBB27D
:1038A0001370654B1B78002B6CD1644B1B78002B7D
:1038B00068D1634B1A6801321A601A68FA235B00F8
:1038C0009A4255D14A4B00221A700421597001398D
:1038D0009970DA7001321A7108325A7145498022A2
:1038E00012048B691342FCD10020FCF7F9FC414B18
:1038F000D96810220A43DA60D96820220A43DA60C4
:10390000D96808220A43DA60394B5B78012398466C
:103910000126384C80252D04354F00239946A36994
:103920002B42FCD14346FB5CDBB223604346F85C90
:10393000029B5840C0B2FCF74BFC029043464A46FB
:10394000FA540136F6B2B0467B7801339E42E6DD8A
:103950002849802212048B691342FCD1254B029A1C
:103960001A60012322490022CA5401333C2BFBD1A7
:10397000334B1A68334B9A4204D901232E4A1370F1
:10398000314A13702D4B1B78002B00D091E11D4B59
:103990001B78002B00D0F4E014490B78DBB25A1CE2
:1039A000D2B20A70032B00D8EBE000230B701F4A41
:1039B0001370264A13780133DBB213701378DBB22D
:1039C000202B00D9C2E01378DBB21F2B00D9D8E03E
:1039D00013785A00D3189B001D4AD3189B7ADB0733
:1039E00040D41A490C001000A7E0C046740600201D
:1039F000FC0200200000154094420050BC0600204C
:103A0000BD08002098010020BF08002014010020FC
:103A1000BC010020FD010020B10100200000054094
:103A20008C000020BB01002020000140290600205E
:103A30003C030020BC08002048030020F8020020BE
:103A4000940100203075000041030020A7040020ED
:103A5000A804002023785A00D3189B00C3189B7A2F
:103A6000DB076AD5B9480378DBB2B9495C00E218D4
:103A700092008A1813890133138103785A00D318EE
:103A80009B00CB181A89C3235B009A4231D103787B
:103A90005A00D3189B00CB189A7A0124A2439A7239
:103AA00003785A00D3189B00CB1800221A81A94B27
:103AB0001A70A94B1B78002B0BD0A84B1B78002B3E
:103AC00007D00078C0B2FDF7CFF90022A44B1A70DE
:103AD00057E09E4B1A789E4851008A18920082182F
:103AE000002191721B785A00D3189B00C3185960AB
:103AF00047E0964C23780133DBB29A4A1370107872
:103B0000C0B2FCF7EDFB23785A00D3189B00904A13
:103B1000D3189B7A5B0734D58F4B1B78002B30D0A2
:103B20008E4B1B78002B2CD0884B1878C0B2FDF739
:103B30009BF900228A4B1A7023E00B780133DBB229
:103B40000B700B78DBB21F2B84D91AE0814B1B78EA
:103B5000002B0ED18449802212048B691342FCD1C0
:103B60007E20FCF7BDFB814A11684B424B4113603C
:103B700004E00123794A13707D4A1370FF22734BCE
:103B80001A707C4B1B78002B0AD07B4B1B88DB0404
:103B900003D50122794B1A6002E00022774B1A60AC
:103BA000774A13780133DBB213701378002B37D1C7
:103BB000744B1B68002B05D1734A13780133DBB2B9
:103BC000137002E00022704B1A706F4B1B78022BAF
:103BD00026D1684B1B78002B03D00022654B1A704E
:103BE00002E00122634B1A70684AFE231370FA3B0D
:103BF00053700023937066480378DBB2591CC9B236
:103C00000170D370872313715A4B1B78591E8B4157
:103C1000DBB25371FCF79AFB5E4B1870FCF732FB7A
:103C20005D4A13780133DBB213705C4B1B68002BC9
:103C300007D15B4B1B68002B03D15A4B1B68002B31
:103C400037D059490B889BB25A1C92B20A80574A06
:103C500093422ED90122564B1A70564A13780133DB
:103C6000DBB213700021504B19801378DBB2092BA3
:103C70001FD90022494B1A60494B1A60494B1A6000
:103C80004C4B1A70414BFE311970FA3959709A70C9
:103C90003F480278D2B2511CC9B20170DA70862254
:103CA0001A71563A5A71FCF751FB3A4B1870FCF7EF
:103CB000E9FA414B1B68002B26D03F4B1A68013AAA
:103CC0001A601B68002B1FD13C4B1B78002B1BD0AC
:103CD00000213B4B984600223A4B9C463A4F3B4EC4
:103CE0003B4D3C4C354B99464B0040461A52604682
:103CF0001A52DA539A535A531A530131C9B24B46E6
:103D00001B78DBB28B42EFD8334B1B78002B00D1F2
:103D100012E1324B1B78002B00D107E1304B1B78AE
:103D2000DBB2532B60D002D84D2B05D0FBE06D2BBE
:103D300002D0732B58D0F6E001222A4B1A706C3255
:103D4000124B1A70FCF79AFBEDE0C046A704002066
:103D5000A8040020B2010020A50400204803002090
:103D6000FE010020FD010020000015406C420050C3
:103D7000410300204B0300203C03002094420050EC
:103D800040030020904200502F060020BC0100207C
:103D9000BB010020B1010020BC080020040200206B
:103DA000880000209C01002000020020B80B0000C9
:103DB00030060020770600208000002099010020B6
:103DC000540100207C06002064030020D000002065
:103DD0003406002008020020F80200207D000020A8
:103DE000480200203E030020AB4B1B78002B57D02D
:103DF000AA494B78303B1B01DBB2A94A13708B7880
:103E00001178303BCB18DBB213701378DBB2202B68
:103E100002D92022A24B1A70A049CB78303B1B015B
:103E2000DBB29F4A53700B795178303BCB18DBB231
:103E300053705378DBB2202B02D92022984B5A7052
:103E400096494B79303B1B01DBB2954A93708B79D5
:103E50009178303BCB18DBB293709378DBB2202B98
:103E600002D920228E4B9A708D490A784B78897836
:103E70009B18CB18DBB28B4D2B708B4C73232370AC
:103E800028780009FCF79AF960702878C0B2FCF72E
:103E900095F9A0700D23E3700422844B1A7035E06D
:103EA0007E4A5178C9B27E4B19709178C9B2597067
:103EB000D278D2B29A701B78DBB2202B02D92022A2
:103EC000774B1A70764B5B78DBB2202B02D920221D
:103ED000734B5A70724B9B78DBB2202B02D9202295
:103EE0006F4B9A706E490A784B7889789B18CB187B
:103EF000DBB26C4A13706C4B732119701278D2B21A
:103F00005A700D229A700A3A684B1A70FCF784F9BD
:103F10000122674B1A706832634B1A70FCF7AEFAD5
:103F200000225E4B1A700022624B1A705F4B1B78A6
:103F3000002B01D0FCF770F95F4B1B78DBB20A2B2A
:103F400000D986E29B005D4AD3589F46554B1B78AB
:103F5000002B02D101225A4B1A700022594B1A70C1
:103F6000574B1B78002B64D1574A916822330B437F
:103F700093600122554B1A600022554B1A70554B25
:103F80001B78002B05D0474B1A780023002A05D157
:103F900048E0514B1B78002BF5D143E04F4A904647
:103FA0004F4A94464F48504F504E514D1A005900B9
:103FB00044460C5BA2466446095B894651466C4602
:103FC000A180A188494505D00178894601214C4648
:103FD000214301705100CC5B895B8946211C6C46F2
:103FE000A180A188494507D03E4909788946022128
:103FF0004C4621433B4C21705200515B3D4C125BBF
:1040000091468AB24A4506D036490A78914604223A
:104010004C4622430A700133DBB2224A1278D2B2F4
:104020009A42C3D8244A13780133DBB21370FFF7E6
:1040300018F80622204B1A70FFF713F8244B1B7850
:10404000002B01D1FFF70DF81F4A916844230B4361
:1040500093600122284B1A60224B1B78002B03D15E
:10406000264B1B78002B0DD01B4B1B78002B02D04E
:1040700069220D4B1A70FCF701FA00231F4A1370D6
:10408000184A13700022124B1A700B4A137801332E
:10409000DBB21370FEF7E5FFCD00002048020020E0
:1040A000B801002099010020BC010020B1010020CE
:1040B0003E0300207D00002049030020D44C000076
:1040C000B3010020BE080020804000508442005010
:1040D000BC080020A5040020F80200207C06002077
:1040E00054010020B4010020D0000020640300200F
:1040F00008020020340600208842005030060020CC
:10410000E44B1B78DBB2032B01D8FEF7AAFFE24A8F
:10411000936844218B4393600023E04A1360DD4A97
:104120001370DF4B1B78002B2BD00022DD4DDE4BB4
:104130009846DE4CDE4B9C46DE48DF4B9A4600211B
:1041400053005E5B6F46BE80BE88B14646464F4612
:104150009F531E5B6F46BE80BE88B14666464F4683
:104160009F531E5A6F46BE80BE885746DE53595332
:10417000195319520132D2B2C94B1B78DBB29342A8
:10418000DED8CE4B1B68002B08D0CD4B1B78C54921
:104190005B00585A8022120202435A52C94B1B68D4
:1041A000002B08D0C64B1B78C0495B00585A8022B0
:1041B000120202435A52C44B1B68002B08D0C04B5A
:1041C0001B78BC495B00585A8022120202435A52A3
:1041D000BE4A13780133DBB21370FEF742FFAD4BDA
:1041E0001B78002B01D1FEF73CFFAB4A91681123ED
:1041F0000B4393600122B64B1A600022A54B1A7044
:10420000B24A13780133DBB21370FEF72AFFA14BD9
:104210001B78002B01D1FEF724FF9F4A93681121E0
:104220008B4393600023AA4A13609A4A1370A74AEB
:1042300013780133DBB21370FEF713FF954B1B7835
:10424000002B01D1FEF70DFF934A936822218B4387
:10425000936000239F4A13608E4A137008229B4B81
:104260001A70FEF7FEFE8B4B1B78002B01D1FEF778
:10427000F8FE894A916844230B4393600122874BDF
:104280001A600022834B1A70904A13780133DBB214
:104290001370FEF7E6FE7F4B1B78DBB2012B01D8D3
:1042A000FEF7DFFE7C4A936844218B439360002035
:1042B0007A4B1860824A13787A4C5B00195B490884
:1042C00019531378794C5B00195B4908195313781B
:1042D00078495B005A5A52085A526E4B1870774B05
:1042E0001B68002B08D0764B1B786E495B00585A30
:1042F0008022120202435A52724B1B68002B08D0D4
:104300006F4B1B7869495B00585A802212020243A6
:104310005A526D4B1B68002B08D0694B1B786549BE
:104320005B00585A8022120202435A52674A13789D
:104330000133DBB21370FEF794FE564B1B78002B53
:1043400001D1FEF78EFE544A916844230B439360DB
:104350000122524B1A6000224E4B1A705B4A1378AE
:104360000133DBB21370FEF77CFE4A4B1B78DBB2E5
:10437000012B01D8FEF775FE474A936844218B4311
:1043800093600020454B18604D4A1378454C5B0004
:10439000195B490819531378444C5B00195B4908B1
:1043A0001953137843495B005A5A52085A52394BF1
:1043B0001870424B1B68002B08D0414B1B783949C1
:1043C0005B00585A8022120202435A523D4B1B682E
:1043D000002B08D03A4B1B7834495B00585A802296
:1043E000120202435A52384B1B68002B08D0344B40
:1043F0001B7830495B00585A8022120202435A52FD
:1044000035490B78DBB25A1CD2B20A700D2B04D896
:1044100008222E4B1A70FEF724FE2C4A1378013323
:10442000DBB21370FEF71DFE1A4B1B78002B01D177
:10443000FEF717FE0022174B1A70214A137801333A
:10444000DBB21370214A13780133DBB21370FEF72D
:1044500008FE104B1B78002B01D1FEF702FE184B13
:104460001B780F4A1278DBB2934202D30022144B1E
:104470001A700022154B1A70FEF7F3FD0023174A3D
:104480001370174A1370174A1370174A1370FFF707
:10449000EBF9C046BC080020804000508842005024
:1044A00099010020540100207C06002064030020B4
:1044B000D000002034060020080200204C420050AA
:1044C000B30100205C4200508C42005049030020A0
:1044D0008042005084420050BE080020BD080020E9
:1044E00098010020BF0800202906002000232E4A42
:1044F00013702E4A13702E4A13702E4A1370FFF752
:10450000B3F92B4A13780133DBB213702A4B1B79B2
:10451000DBB2F02B01D0FFF720F9FEF78BFF002470
:10452000264D63001A199200AA18907A04210843B4
:104530000121014391720027002111811E494E790A
:10454000F6B21B199B005E558D79EDB25570C87996
:10455000C0B290700B7A13714B7A53718B7A93714E
:10456000C97ACBB29846D371154B1F700C21597084
:104570000B219970DF701F7170275F71671CFFB28C
:104580009F71DE711D725872107998725079D872CD
:1045900092791A7342465A730A4B1B78002B01D149
:1045A000FEF7C5FFFEF7AEFFBD0800209801002012
:1045B000BF0800202906002014010020A8040020C4
:1045C000FC020020A504002010B5354B1B68DBB2AF
:1045D000344A1278D2B21F2A09D8324A1278013AE4
:1045E00051008A18920030498A18002111812F4AFF
:1045F0001278002A23D1012B51D901212B4A1170A5
:104600002B490A789BB202329A18FF2002402948AF
:1046100002800A78D2B2501CC0B2087026485200FC
:104620008024640014520A78D2B2541CE4B20C7094
:10463000520013520B785B0000221A522FE01C4AE2
:1046400012781C490988914219D10024174A147024
:1046500017490A78D2B2501CC0B208709BB21648F3
:10466000520013520B78DBB25A1CD2B20A705B00B4
:10467000802292001A520B785B001C520FE00C490A
:104680000A78D2B2501CC0B208709BB20A485200DD
:1046900013520B785B0000221A52084B1A7010BD9F
:1046A00000001540FD010020A80400209801002012
:1046B000BD08002074000020BC0600202906002050
:1046C000F0B583B0634B1B68DBB26A46D371624BB3
:1046D0001B78002B00D1AAE0604B9B78002B17D0F1
:1046E000012B00D0B3E05D4BD9784A1CDA706B46E1
:1046F000DA1DDB79DBB25A48435413780D2B00D016
:10470000A5E00022554B9A700132564B1A709EE07C
:104710006B4607331B784D3BDAB2292A00D996E065
:104720009300514AD3589F46504A514B1A60012278
:104730004A4BDA706B4607331B78DBB248490B7083
:10474000484B1A7083E0494A494B1A600123494A91
:1047500013704249CB706A4607321278D2B2404891
:1047600002708B7073E0444A137859424B41DBB2BC
:1047700013707421414B197013785A1E93413033D2
:104780003E4A53700D23937003223D4B1A705EE036
:104790003A4B56221A706521597072209870283A47
:1047A000DA7031241C715A7130259D71DC71023C24
:1047B0001C7213345C7239359D724426DE721D738F
:1047C0005C73153C9C730A35DD730C3E1E745E747D
:1047D0009C741C34DC7425341C7506345C75997526
:1047E000D8750C38187629365E7603389876D976DF
:1047F000453919774C3C5C7798773A38D877542705
:104800005F54333FDE554C373F3E9F5501369D5533
:104810004F3D5955213505315D54273501315D54E2
:1048200001315A54213A1A55154B18700FE0154AA8
:104830001378DBB2591CC9B2117069460731097887
:10484000C9B21148C1541378DBB20022C25403B07C
:10485000F0BDC04600000540F802002074000020B2
:10486000480200207D000020104D0000A0860100BD
:104870008000002076060020CD000020BC01002032
:10488000B101002084000020A403002010B582B0F4
:104890000422204901A800F023F91F4B1B6A0020C5
:1048A000A022D202134216D11A0301D41B4800E001
:1048B0001B489A030FD4DA05D20D02328008504308
:1048C0001A04920F01A9895C9B04DB0E0233594341
:1048D00000F07AF88000134B18600F4B1B69072219
:1048E0001340022B03D09B000A4AD31858680A4B86
:1048F0009B690F211940013100F066F8094C606096
:10490000094B9C466044094900F05EF8A06002B083
:1049100010BDC046B84D000000020050001BB7009B
:10492000008051010000002020A1070040420F003C
:1049300030B500221E4B1A601E4B1B690732134014
:104940000DD11D4A1B4B1A621C4B1A48042102E070
:10495000013B002B23D0C2681142F9D01FE0072B86
:1049600025D1174A134B1A62164B1248042102E054
:10497000013B002B13D0C2681142F9D00FE0D55093
:10498000D450D050D1580029F9D00222094B1A61D5
:10499000002180235B00A022D205D15007E0A02295
:1049A000D20580235B00592516248820E7E730BD17
:1049B000000000200002005017420000E12E00001D
:1049C0003956080067560000002243088B4274D312
:1049D00003098B425FD3030A8B4244D3030B8B4200
:1049E00028D3030C8B420DD3FF22090212BA030C09
:1049F0008B4202D31212090265D0030B8B4219D3EA
:104A000000E0090AC30B8B4201D3CB03C01A524109
:104A1000830B8B4201D38B03C01A5241430B8B4251
:104A200001D34B03C01A5241030B8B4201D30B033A
:104A3000C01A5241C30A8B4201D3CB02C01A524161
:104A4000830A8B4201D38B02C01A5241430A8B4224
:104A500001D34B02C01A5241030A8B4201D30B020D
:104A6000C01A5241CDD2C3098B4201D3CB01C01A27
:104A7000524183098B4201D38B01C01A5241430931
:104A80008B4201D34B01C01A524103098B4201D31F
:104A90000B01C01A5241C3088B4201D3CB00C01A8C
:104AA000524183088B4201D38B00C01A5241430804
:104AB0008B4201D34B00C01A5241411A00D2014629
:104AC000524110467047FFE701B5002000F006F89C
:104AD00002BDC0460029F7D076E770477047C04650
:104AE00070B50F2A32D90C0004430B00A40731D152
:104AF00015000400103D2D0901352D0149191E68CE
:104B000026605E6866609E68A660DE681033E660B8
:104B100010349942F3D10F2345191340032B1BD9AD
:104B20001C1F0023A4080134A400CE58EE50043307
:104B30009C42FAD103232D1909191A4005D00023EC
:104B4000CC5CEC5401339A42FAD170BD0500002AC6
:104B5000F5D1FAE70500F2E71A00F8E73C1C00007F
:104B60003C12000020150000F6150000EE150000B4
:104B70004A15000096150000C41500001A17000021
:104B80008A1B0000621700007A1200001C1300004C
:104B90006C1200005C1B00003C1C000006160000AC
:104BA00050160000321600003C1C0000DA1900000C
:104BB000B019000088170000B8180000C81B0000DA
:104BC000AA1A00002A1200003C1C00003C1C000035
:104BD0003C1C00003C1C00003C1C00003C1C000075
:104BE0003C1C00003C1C00003C1C00003C1C000065
:104BF0003C1C00003C1C00003C1C00003C1C000055
:104C00003C1C00003C1C00003C1C00003C1C000044
:104C10003C1C00003C1C00003C1C0000C01B0000B1
:104C2000C01B0000B4290000F41C00002A1D000075
:104C3000641D00005A1D00006E1D0000C81D00000C
:104C4000541E0000841E0000B4290000D21E000083
:104C5000B4290000B4290000B4290000B4290000E0
:104C6000B4290000E6230000BE2400002024000038
:104C7000D4260000B4290000B4290000B4290000A3
:104C8000B4290000B42900005C220000FE1E0000D0
:104C9000B4290000B4290000B4290000B4290000A0
:104CA000B4290000E6270000582900005829000018
:104CB00058290000B42900002A2900004C250000D2
:104CC00082250000C0250000F625000034260000E3
:104CD0006A2600004C3F00003C40000000410000FC
:104CE000DE4100000E4200003C420000664200002F
:104CF000964200003A4300006A4300002844000046
:104D0000001BB700000000000000000000805101FF
:104D1000284700004E4800004E4800004E48000062
:104D20004E4800004E48000046470000664700001D
:104D30004E480000904700004E4800004E480000DA
:104D40004E4800004E4800004E4800004E4800000B
:104D50004E4800004E4800004E4800004E480000FB
:104D60004E4800004E4800004E4800004E480000EB
:104D70004E4800004E4800004E4800004E480000DB
:104D80004E4800004E4800004E4800004E480000CB
:104D9000284700004E4800004E4800004E480000E2
:104DA0004E4800004E48000046470000664700009D
:104DB0004E4800009047000001020204001BB700AB
:104DC0000000000080F0FA02102700000000000040
:0C4DD00000000000000000000080510105
:0C4DDC0080F0FA0280F0FA0232000000C1
:00000001FF
